:10000000EFEF02F00000000000EF00F00000000041
:0A0010000000000000000000F3D71C
:10001C00240E0C6EB50E0D6E0D2EFED70C2EFCD7CD
:06002C00000000001200BC
:0A003200530E0D6E0D2EFED71200C6
:0C003C00000000000000000000001200A6
:1000480001017FBF02D08A9A01D08A8A7FBD02D07F
:100058008A9801D08A887FBB02D08A9601D08A8686
:100068007FB902D08A9401D08A84000190B102D06D
:100078008A8001D08A908A82DDDF8A9201017FB767
:1000880002D08A9A01D08A8A7FB502D08A9801D094
:100098008A887FB302D08A9601D08A867FB102D03F
:1000A8008A9401D08A84000190B102D08A8001D05C
:1000B8008A908A82BFDF8A9290A102D0ABDF01D0FA
:0400C800B4DF12008F
:1000CC00AECF02F0ABA202D0AB98AB8802C001F06D
:0600DC0001C000F012005B
:1000E200086A080E0C6E003408360450085ED8B058
:0E00F20002D00826D89000360C2EF5D712004A
:0E010000000190917CC17FF19FDF9081120081
:0E010E00000E9EBA010E016E01C000F012003C
:10011C00086A096A100E0C6E013408360936045050
:10012C00085E0550D8A0053C095ED8B007D0045035
:10013C0008260550D8B0053C0926D8900036013663
:06014C000C2EEAD71200A0
:1001520001017C51010A03E1800E7C6F14D07C51B5
:10016200020A03E1C00E7C6F0ED07C51030A03E148
:10017200940E7C6F08D07C51040A03E1D40E7C6F8C
:1001820002D0800E7C6F7D05006E7C51002600C07F
:100192007CF10001908100C07FF155DF90917EC11A
:0801A2007FF151DF9081120092
:0C01AA00240E0D6E0D2EFED7000012007A
:1001B60077C1E1FF78C1E2FF200EE66E200EE66E03
:1001C600300EE66EE66A020E01017725796F000EA3
:1001D60078217A6F7651000A1AE00A0E046E76C10B
:1001E60000F07CDF08C000F079C1E1FF7AC1E2FFD0
:1001F600300E0024E66E0A0E046E76C100F06EDF45
:1002060000C076F1010E795F000E7A5BE3D712002B
:100216000001DC6BDC510101775D1FE30001DC515D
:1002260001017825E16E000E7921E26E0001DC51B4
:1002360001017625006EDD0EE96E000EEA6E0050B5
:10024600E926D8B0EA2AEECFE6FF0001DC5101012B
:10025600771903E00001DC2BDDD701017751782502
:0E026600E16E000E7921E26E000EE66E1200CF
:1002740001017651010A03E1800E766F14D07651A4
:10028400020A03E1C00E766F0ED07651030A03E131
:10029400940E766F08D07651040A03E1D40E766F7B
:1002A40002D0800E766F7705006E7651002600C06E
:1002B40076F100C07FF1C6DE909101017A6B7A512C
:1002C4007825E96E000E7921EA6EEE50000A0CE002
:1002D4007A517825E96E000E7921EA6EEECF7CF131
:0E02E4000DDF01017A2BEBD700019081120093
:1002F2000900F5CFE6FF0006FBE10106F9E1120075
:10030200FF0E0001996FFF0E9A6FFF0E9B6FFF0E9B
:100312009C6FCC0E9D6F000E9E6F000E9F6F000EA5
:10032200A06F0E0E916F010E926F000E936F000E72
:10033200946FFF0E956FFF0E966F000E976F000E73
:10034200986FAC8A900EAB6E948E949C9EAA03D04A
:08035200AECF00F0FBD7120052
:10035A00FF0E00018C6FFF0E8D6FFF0E8E6FFF0E6A
:0E036A008F6FC26A070EC012C08EC2801200D2
:1003780093929390939493969398939A8A928A904F
:100388008A9A8A988A968A9445DE44DE43DE8A866B
:100398008A848A824FDE8A923DDE8A824BDE8A9286
:1003A80039DE8A8247DE8A9235DE8A948A8242DE84
:1003B8008A9230DE8A823EDE8A928A968A8A8A8287
:1003C80039DE8A9227DE8A9A8A848A8233DE8A9282
:1003D8008A948A822FDE8A921DDE8A822BDE8A9296
:1003E8008A848A8227DE8A9215DE8A948A8222DEAD
:1003F8008A928A8A8A888A868A848A821BDE8A9274
:0804080009DE000190811200E1
:10041000480E01017F6F18DE0101786B1C0E7825F4
:10042000F66E130EF76E000EF722000EF86E000E39
:10043000F8220900F5CF7CF163DE01017851070A4B
:1004400002E0782BEBD7020E7F6FFEDD76C17CF1E8
:0E04500077C17DF1010E01017E6F7BDE12008F
:10045E0057DE0050010AFCE132DE00C076F176C1B3
:04046E0000F0120088
:1004720078C1E1FF79C1E2FF300EE66E300EE66E22
:10048200300EE66E300EE66E300EE66EE66A040E52
:10049200010178257A6F000E79217B6F000E7719A2
:1004A20002E1000E761927E00A0E046E000E056EB8
:1004B20076C100F077C101F030DE08C000F009C05B
:1004C20001F0300E00267AC1E1FF7BC1E2FF00C0DD
:1004D200E6FF0A0E046E000E056E76C100F077C1CB
:1004E20001F01BDE00C076F101C077F1010E7A5FE8
:0804F200000E7B5BD3D7120062
:1004FA00500E01017F6FA3DD0101786B0C0E782588
:10050A00F66E130EF76E000EF722000EF86E000E4E
:10051A00F8220900F5CF7CF1EEDD01017851070AD6
:10052A0002E0782BEBD7020E7F6F89DD76C17CF172
:0E053A0077C17DF1020E01017E6F06DE120018
:10054800400E01017F6F7CDD0101786B140E782568
:10055800F66E130EF76E000EF722000EF86E000E00
:10056800F8220900F5CF7CF1C7DD01017851070AAF
:1005780002E0782BEBD7020E7F6F62DD76C17CF14B
:0C05880077C17DF101017E6BE0DD120007
:10059400C26A070EC012C08E76C100F00036009009
:1005A400003600900050C212C280FDDDC282C2A299
:1005B40002D00000FCD7C4CF01F0006A00C077F17C
:1005C40001C078F1C35001017713000E7813C29073
:0A05D40077C100F078C101F01200B9
:1005DE00B886040EB06E110EAF6EAC848BDE030EB9
:1005EE000B6E8A0E0C6E550E0D6E0D2EFED70C2E4A
:1005FE00FCD70B2EFAD700000000929A92949480AA
:10060E0094829484010EC26E010EC16E9FDE92948E
:10061E00928A200E01014A6F470E4B6F450E4C6FAA
:10062E004E0E4D6F450E4E6F520E4F6F410E506F68
:10063E00540E516F450E526F550E536F520E546F2E
:10064E00200E556F310E566F300E576F200E586FAD
:10065E004D0E596F480E5A6F7A0E5B6F200E5C6FFF
:10066E00200E5D6F5E6B530E356F590E366F4E0E4C
:10067E00376F430E386F480E396F520E3A6F4F0E6A
:10068E003B6F4E0E3C6F490E3D6F530E3E6F450E47
:10069E003F6F200E406F500E416F410E426F520E53
:1006AE00436F200E446F470E456F500E466F530E2C
:1006BE00476F200E486F496B200E206F520E216F30
:1006CE004F0E226F430E236F4B0E246F570E256F66
:1006DE00450E266F4C0E276F4C0E286F200E296F7D
:1006EE004A0E2A6F550E2B6F500E2C6F490E2D6F22
:1006FE00540E2E6F450E2F6F520E306F200E316F2F
:10070E00200E326F200E336F346B200E5E6E540E41
:10071E005F6E550E0001606F330E616F300E626FAB
:10072E002D0E636F440E646F310E656F340E666F5F
:10073E00300E676F200E686F760E696F320E6A6F1D
:10074E002E0E6B6F330E6C6F300E6D6F200E6E6F44
:10075E00200E6F6F200E706F200E716F726B05DEA4
:10076E00010E01017F6F69DC0C0E01017F6F65DCEC
:10077E00010E0101766F010E776F4A0E786F010E32
:10078E00796F71DD020E0101766F010E776F350EF6
:10079E00786F010E796F67DD030E0101766F010E22
:1007AE00776F200E786F010E796F5DDD040E0101FB
:1007BE00766F010E776F5E0E786F000E796F53DDD8
:1007CE00CB0E0B6EEC0E0C6E840E0D6E0D2EFED738
:1007DE000C2EFCD70B2EFAD70000010E736F560E9F
:1007EE005C6E5D6A010E756F300E766F300E776F30
:1007FE00786B82B204D000012E0E746F03D000010C
:10080E002F0E746F25DE00C0DCF00050240A01E0CC
:10081E00F9D70001DC6BDD0E0101746F000E756FF0
:10082E000001DC5101017427D8B0752B11DE74C1A3
:10083E00E1FF75C1E2FF00C0E6FFDD0EE96E000EBE
:10084E00EA6E0001DC51E926D8B0EA2AEE502A0AF7
:10085E0002E1DC6B01D0DC2BDC51000AFF0ED8A4C8
:10086E00000E016EDC51420AFF0ED8A4000E006E7F
:10087E000150001201E1CFD77351010AD8A499D0CB
:10088E00DF51520AFF0ED8A4000E016EE0514D0A40
:10089E00FF0ED8A4000E006E00500116E151430A5F
:1008AE00FF0ED8A4000E006E01500016D8B481D0F1
:1008BE00020E736F010E5D6E5CC0DCF0EAC05CF080
:1008CE00EA51DC1905E0010E01017F6F24EC00F006
:1008DE005C50410A6EE19284929A060E0101766F87
:1008EE00060E776F2B0E786F000E796F8DDC300E43
:1008FE002B5C006E0A0E0002F3CF00F02C50002687
:10090E0000017451005E00C0DCF000C076F1360EBE
:10091E000101776F000E786F47DC0F0E766F020EB7
:10092E00776F150E786F000E796F6EDC110E766F85
:10093E00020E776F200E786F000E796F65DC140E45
:10094E00766F040E776F500E786F000E796F5CDC49
:10095E00F6C05BF01B0E766F030E776F3A0E786F54
:10096E00000E796F51DC1E0E766F020E776F450EFC
:10097E00786F000E796F48DC210E766F040E776F5C
:10098E00810E786F000E796F3FDC03C1B7F0280E31
:10099E00766F040E776FB80E786F000E796F34DCB9
:1009AE00320E766F060E776FA10E786F000E796F8E
:1009BE002BDC00017351020A3FE1DF51470AFF0EA3
:1009CE00D8A4000E016EE051470AFF0ED8A4000E07
:1009DE00006E00500116E151410AFF0ED8A4000E20
:1009EE00006E0150001628E0010E736F010E5D6E51
:1009FE005C50410A21E19284929A280E0101766F91
:100A0E00020E776F760E786F000E796F0BEC01F099
:100A1E002B0E766F040E776FAC0E786F000E796F1B
:100A2E000BEC01F0300E766F050E776FCF0E786FF0
:100A3E00000E796F0BEC01F00101766BA4DD00C0A6
:100A4E0002F001C003F003320232039E02C0DAF05C
:100A5E0003C0DBF002C076F103C077F1C30E786FEE
:100A6E00000E796FFFDC010E766F8DDD00C002F097
:100A7E0001C003F003320232039E02C0DAF003C05B
:100A8E00DBF002C076F103C077F1C90E786F000E6D
:100A9E00796FE8DC5D50010AD8A483EF09F082B0CB
:100AAE001AD00001752B070E0B6E580E0C6E590ED8
:100ABE000D6E0D2EFED70C2EFCD70B2EFAD7000086
:100ACE0000007551030A02E1010E756F010E01015E
:100ADE007F6F24EC00F05C50560AD8A4D3D09294C9
:100AEE00928A010E0101766F010E776F200E5F6FF5
:100AFE00200E606F200E616F200E626F200E636FEE
:100B0E00450E646F4E0E656F200E666F410E676F59
:100B1E00540E686F540E696F450E6A6F4E0E6B6FF2
:100B2E00540E6C6F450E6D6F200E6E6F200E6F6F34
:100B3E00200E706F200E716F200E726F736B5F0E32
:100B4E00786F010E796F3AEC01F0020E0101766FAB
:100B5E00010E776F200E5F6F200E606F200E616F9B
:100B6E00200E626F200E636F200E646F200E656F75
:100B7E00200E666F200E676F440E686F450E696F0C
:100B8E00200E6A6F200E6B6F200E6C6F200E6D6F35
:100B9E00200E6E6F200E6F6F200E706F200E716F15
:100BAE00200E726F736B5F0E786F010E796F3AECD9
:100BBE0001F0030E0101766F010E776F200E5F6F4D
:100BCE00200E606F200E616F540E626F520E636FB7
:100BDE00410E646F4D0E656F450E666F530E676F57
:100BEE00200E686F560E696F410E6A6F4C0E6B6F5A
:100BFE00490E6C6F440E6D6F450E6E6F530E6F6F18
:100C0E00200E706F200E716F200E726F736B5F0E61
:100C1E00786F010E796F3AEC01F0040E0101766FD8
:100C2E00010E776F200E5F6F200E606F200E616FCA
:100C3E00200E626F200E636F200E646F200E656FA4
:100C4E00200E666F200E676F200E686F200E696F84
:100C5E00200E6A6F200E6B6F200E6C6F200E6D6F64
:100C6E00200E6E6F200E6F6F200E706F200E716F44
:100C7E00200E726F736B5F0E786F010E796F3AEC08
:100C8E0001F039D300017551010AD8A4C1D1010E6A
:100C9E000101766F010E776F4C0E5F6F610E606F04
:100CAE00740E616F200E626F3A0E636F200E646FCA
:100CBE00200E656F666B5F0E786F010E796F3AECE2
:100CCE0001F0010E0101766F080E776F150E786F29
:100CDE00000E796F3AEC01F0010E01017C6F0A0EE5
:100CEE007D6FDF0E7E6FA9EC00F0010E0101766FB5
:100CFE000B0E776F200E786F000E796F3AEC01F0C5
:100D0E00010E01017C6F0D0E7D6F2E0E7E6FA9EC14
:100D1E0000F0010E0101766F0E0E776F500E786F98
:100D2E00000E796F3AEC01F0010E01017C6F120E8C
:100D3E007D6F200E7E6FA9EC00F0010E01017C6F1D
:100D4E00130E7D6F5BC07EF1A9EC00F0020E010167
:100D5E00766F010E776F4C0E5F6F6F0E606F6E0EBB
:100D6E00616F200E626F3A0E636F200E646F656BBB
:100D7E005F0E786F010E796F3AEC01F0020E0101F1
:100D8E00766F070E776F3A0E786F000E796F3AEC2A
:100D9E0001F0020E01017C6F0A0E7D6FDF0E7E6F79
:100DAE00A9EC00F0020E0101766F0B0E776F450E67
:100DBE00786F000E796F3AEC01F0020E01017C6F34
:100DCE000D0E7D6F2E0E7E6FA9EC00F0020E01014E
:100DDE00766F0E0E776F810E786F000E796F3AEC8C
:100DEE0001F0020E01017C6F120E7D6F200E7E6FE0
:100DFE00A9EC00F0020E01017C6F130E7D6FB7C0DF
:100E0E007EF1A9EC00F0020E01017C6F140E7D6FD5
:100E1E00200E7E6FA9EC00F0030E0101766F010E1D
:100E2E00776F410E5F6F6C0E606F740E616F200EE8
:100E3E00626F3A0E636F200E646F656B5F0E786F94
:100E4E00010E796F3AEC01F0030E0101766F070E79
:100E5E00776FCF0E786F000E796F3AEC01F0030EBC
:100E6E000101766F0A0E776F7DEC02F0030E010121
:100E7E00766F0C0E776F200E5F6F6D0E606F650EC6
:100E8E00616F740E626F720E636F650E646F730E18
:100E9E00656F200E666F200E676F686B5F0E786F42
:100EAE00010E796F3AEC01F0030E0101766F0E0E12
:100EBE00776FA4EC02F0040E01017C6F010E7D6FC2
:100ECE00A1C07EF1A9EC00F0040E01017C6F020EB0
:100EDE007D6FA2C07EF1A9EC00F0040E0101766FC9
:100EEE00030E776F08EC02F0040E01017C6F040E06
:100EFE007D6FA3C07EF1A9EC00F0040E01017C6FA2
:100F0E00050E7D6FA4C07EF1A9EC00F0040E010168
:100F1E00766F060E776F08EC02F0040E0101766F05
:100F2E00070E776F320E5F6F300E606F616B5F0E64
:100F3E00786F010E796F3AEC01F0040E01017C6FAF
:100F4E00090E7D6FA5C07EF1A9EC00F0040E010123
:100F5E007C6F0A0E7D6FA6C07EF1A9EC00F0040E28
:100F6E000101766F0B0E776F200E5F6F200E606F94
:100F7E00616B5F0E786F010E796F3AEC01F0040E23
:100F8E0001017C6F0D0E7D6F37C07EF1A9EC00F074
:100F9E00040E01017C6F0E0E7D6F38C07EF1A9EC40
:100FAE0000F0040E01017C6F0F0E7D6F3A0E7E6F06
:100FBE00A9EC00F0040E01017C6F100E7D6F2DC0A8
:100FCE007EF1A9EC00F0040E01017C6F110E7D6F15
:100FDE002EC07EF1A9EC00F0040E01017C6F120E02
:100FEE007D6F3A0E7E6FA9EC00F0040E01017C6F4E
:100FFE00130E7D6F2FC07EF1A9EC00F0040E0101DF
:10100E007C6F140E7D6F30C07EF1A9EC00F073D1B1
:10101E007551020AD8A46FD182B454D0010E0101C9
:10102E00766F010E776F540E5F6F650E606F6E0EEA
:10103E00616F730E626F690E636F6F0E646F6E0E6B
:10104E00656F200E666F500E676F490E686F4C0EFF
:10105E00696F450E6A6F3A0E6B6F200E6C6F6D6B7B
:10106E005F0E786F010E796F3AEC01F0010E0101FF
:10107E007C6F0F0E7D6FCBC07EF1A9EC00F0010EE0
:10108E000101766F100E776F7DEC02F0010E0101FB
:10109E007C6F110E7D6FCCC07EF1A9EC00F0010EBD
:1010AE000101766F120E776F200E5F6F560E606F16
:1010BE00200E616F626B5F0E786F010E796F3AECE6
:1010CE0001F034D0010E0101766F010E776F540ED0
:1010DE005F6F650E606F6E0E616F730E626F690EDD
:1010EE00636F6F0E646F6E0E656F200E666F500E1F
:1010FE00676F490E686F4C0E696F450E6A6F3A0E38
:10110E006B6F200E6C6F2D0E6D6F2E0E6E6F2D0E83
:10111E006F6F200E706F560E716F200E726F736BA5
:10112E005F0E786F010E796F3AEC01F0020E01013D
:10113E00766F010E776F540E5F6F650E606F6E0ED9
:10114E00616F730E626F690E636F6F0E646F6E0E5A
:10115E00656F200E666F560E676F430E686F580EE2
:10116E00696F4F0E6A6F3A0E6B6F200E6C6F6D6B60
:10117E005F0E786F010E796F3AEC01F0020E0101ED
:10118E007C6F0F0E7D6FC5C07EF1A9EC00F0020ED4
:10119E000101766F100E776F7DEC02F0020E0101E9
:1011AE007C6F110E7D6FC6C07EF1A9EC00F0020EB1
:1011BE000101766F120E776F200E5F6F560E606F05
:1011CE00200E616F626B5F0E786F010E796F3AECD5
:1011DE0001F0030E0101766F010E776F4E0E5F6FF9
:1011EE00620E606F720E616F650E626F200E636F1E
:1011FE00640E646F650E656F200E666F730E676FFB
:10120E00610E686F740E696F2E0E6A6F3A0E6B6FF9
:10121E00200E6C6F6D6B5F0E786F010E796F3AEC6E
:10122E0001F0030E0101766F0F0E776F760E786F59
:10123E00000E796F3AEC01F0030E0101766F110E7C
:10124E00776F200E5F6F200E606F200E616F200E85
:10125E00626F636B5F0E786F010E796F3AEC01F07F
:10126E00040E0101766F010E776F480E5F6F440E0C
:10127E00606F4F0E616F500E626F3A0E636F200EED
:10128E00646F656B5F0E786F010E796F3AEC01F04B
:10129E00040E0101766F070E776FAC0E786F000E9D
:1012AE00796F3AEC01F0040E0101766F080E776F3C
:1012BE007DEC02F0040E0101766F0B0E776F200E9F
:1012CE005F6F200E606F200E616F200E626F200E1A
:1012DE00636F200E646F200E656F200E666F200EFA
:1012EE00676F200E686F696B5F0E786F010E796FF6
:0E12FE003AEC01F000D05D6A00EF04F0FFD77B
:08130C0000000000000C0408C1
:0813140008040E111F100E0069
:08131C000000000E00000000BB
:020000040030CA
:0E000000000C1F1EFF8381FF0FC00FE00F409A
:00000001FF
